:10000000EE2A00308A000408840A8207003448344B
:1000100065346C346C346F3420344B34693474344C
:100020006334683475342034573465346C34633445
:100030006F346D3465342E342E342E342034003435
:1000400065346C3465346B34743472346F346E34AC
:1000500069346B34733466346F3472346B3469349E
:10006000643473342E3463346F346D34203400348C
:1000700047346F346F34643420344D346F34723409
:0E0080006E3469346E34673420342134003419
:1005DC0083019E2B83128E0085110E08803E06230C
:1005EC0008008312851101300623043083128F001A
:1005FC00E4308E008E0B002B8F0B002B6400080058
:10060C0083128D000D308C008C0B0A2B83120D087D
:10061C008C00043003108C0CFF3E031D102B0C08B7
:10062C000F398600851485100D080F398600851446
:10063C008510080083129100851500308F00003062
:10064C009000372B110884000120062301308312FF
:10065C008E000E08910701308F070318900A0030A6
:10066C009007110884000120003A03193E2B3F2B00
:10067C004C2B1008803ACE0080304E02031D482BC4
:10068C0010300F02031C4B2B4C2B282B0800033073
:10069C008312900010089200831685018601831244
:1006AC008511851005112E30910073309000900B40
:1006BC005D2B910B5D2B14308312910079309000DF
:1006CC00900B662B910B662B6B2B831212088600FA
:1006DC0085148510073091007D309000900B742BA1
:1006EC00910B742B83128514851042309000900B63
:1006FC007D2B640083128514851042309000900B82
:10070C00852B64000230831286008514851003301B
:10071C00910097309000900B912B910B912B962B75
:10072C00283006230C300623F72206300623080057
:10073C004D23013083129600003097000130930056
:10074C00130899001A309300130898000030F02217
:10075C008312190820238312180820234030F0221A
:10076C003230202302308312950044309400A9309B
:10077C009300930BBF2B940BBF2B950BBF2B6400DB
:10078C00823083129400DD309300930BCB2B940BAF
:10079C00CB2BD02B8312190884000120003A0319AB
:1007AC00D82BD92BDE2B0130930013089907FD2B86
:1007BC00170816040319E32BE42BF12B01309300DB
:1007CC00130899001A309300130898000030960013
:1007DC0000309700FD2B1A3093001308990001305C
:1007EC009300130898000130960000309700F72210
:0407FC00AC2B0028FA
:00000001FF
